:100000000C948F000C94AE000C94AE000C94C402BF
:100010000C94AE000C94AE000C94AE000C94AE00A8
:100020000C94AE000C94AE000C94AE000C94AE0098
:100030000C94AE000C94AE000C94AE000C942B1EED
:100040000C94AE000C94AE000C94AE000C94AE0078
:100050000C94AE000C94AE000C94AE000C94AE0068
:100060000C94AE000C94AE000C94AE000C94AE0058
:100070000C94AE000C94AE000C94AE000C94AE0048
:100080000C94AE000C9441070C94AE00770DF30D68
:10009000F30DF30D870D9B0DA20DAB0DB80DF30DF8
:1000A000C60DCD0DC10DD30DF30DF30DF30DFE0DEA
:1000B000F30DF30DF30DF30DF30DF30DF30DDE0D55
:1000C000E50DF30DF30DF30D7F0DF30DF30DF30DB2
:1000D000F30DF30DF30DF30DF30DF30DF30DF30D20
:1000E000F30DF30DEC0D73107F108B109710A31010
:1000F000AF10BC10D410E210F010FE100C111A1149
:100100002A1151115D116911751181118D119A1109
:10011000B211C011CE11DC11EA11F811081211242C
:100120001FBEC0E0D0E1DEBFCDBF11E0A0E0B1E076
:10013000E6EBFFE300E00BBF02C007900D92AC3A84
:10014000B107D9F727E0ACEAB1E001C01D92AC38A5
:10015000B207E1F70E942E140C94D91F0C940000F2
:10016000E199FECF21E0280F2EBB01969FBB6DBB0E
:10017000E29AE19A0895E199FECF21E0280F2EBB83
:1001800001969FBBE09A8DB30895E199FECF1EBA08
:100190001FBA8FEF8DBBE29AE19A0895E199FECFE5
:1001A0001EBA1FBA1DBAE29AE19A0895CF93DF935F
:1001B000C0E7D2E081E0888319821A828B83E091C4
:1001C0007802F091790281818F5F8C83E0917A02CD
:1001D000F0917B029181890F8D831E8268E0CE01B0
:1001E0000E947F1E8F83DF91CF910895CF93DF937D
:1001F00080E390E00E94B81E909379028093780289
:1002000080E090E0E0917802F0917902E80FF91F28
:100210001082019680339105A9F7E0917802F09160
:10022000790281E08083E0917802F091790286E0A2
:100230008183E0917802F091790289E182831382CF
:100240001482158284EC868389E4878390E5908705
:1002500092E3918782878AEC8387A6E7B1E08CE0FE
:1002600090E02D91E0917802F0917902E80FF91F6A
:100270002083019686319105A1F7E0917802F091F3
:10028000790289EC868BA1E8B1E087E190E02D91BD
:10029000E0917802F0917902E80FF91F208301962E
:1002A00080329105A1F7E0917802F091790285EC16
:1002B00080A3A5E8B1E081E290E02D91E091780281
:1002C000F0917902E80FF91F20830196863291059B
:1002D000A1F7E0917802F091790287EC86A3ABE870
:1002E000B1E087E290E02D91E0917802F0917902FF
:1002F000E80FF91F208301968E329105A1F7C09176
:100300007802D091790281EC8EA760E3CE010E9441
:100310007F1E8FA7DF91CF910895CF93DF9380E366
:1003200090E00E94B81E90937B0280937A0280E056
:1003300090E0E0917A02F0917B028033910529F000
:10034000E80FF91F10820196F4CF81E08083E091DD
:100350007A02F0917B0286E08183E0917A02F0914B
:100360007B0289E1828384EC838389E4848390E542
:10037000958392E3968387838AEC8087A6E7B1E032
:1003800089E090E02D91E0917A02F0917B02E80FF4
:10039000F91F2083019683319105A1F7E0917A023C
:1003A000F0917B0285EC838BA5E8B1E0ED0184E15F
:1003B00090E02991E0917A02F0917B02E80FF91F19
:1003C0002083019689319105A1F7E0917A02F0919D
:1003D0007B0282EC818F86E7828F81E3838F85ECBD
:1003E000848F8DE190E02D91E0917A02F0917B0273
:1003F000E80FF91F2083019682329105A1F7E09161
:100400007A02F0917B0280EC82A387EC83A3ABE8B5
:10041000B1E084E290E02D91E0917A02F0917B02CC
:10042000E80FF91F208301968B329105A1F7C09147
:100430007A02D0917B0281EC8BA760E3CE010E940F
:100440007F1E8FA7DF91CF910895CF93DF93CCE7E5
:10045000D2E080EC888382E8898386E08A831B82ED
:100460001C828AE58D8381E38E831F8286E18887E3
:1004700019868AE08A8766E081E892E00E947F1E02
:100480008B8365E0CE010E947F1E8C83DF91CF912C
:10049000089580917802909179020E94501F809176
:1004A0007A0290917B020C94501FEF92FF920F936F
:1004B0001F93CF93DF930E94F6000E948D010E944C
:1004C00025020E94D6001FB7F89480E7E82E82E04C
:1004D000F82EC0E0D0E0F70161917F01CE010E94CB
:1004E000B0002196C830D105B1F7C0E0D0E00C2FA4
:1004F000085FE0917802F0917902818128E0829F83
:10050000C0011124C817D9074CF4EC0FFD1F6081FE
:10051000802F90E00E94B0002196E9CFC0E0D0E0AB
:100520008C2F800FE0917A02F0917B02218198E07C
:10053000299F90011124C217D30744F4EC0FFD1F2B
:10054000608190E00E94B0002196EACFCCE7D2E033
:1005500020917E0230E02C5F3F4FAE014C5752405D
:100560002417350744F0699101E0080F90E00E94DC
:10057000B000802FEDCF1FBFDF91CF911F910F9162
:10058000FF90EF900C9449021F920F920FB60F92BA
:1005900011240BB60F922F933F934F935F936F935A
:1005A0007F938F939F93AF93BF93EF93FF9310929B
:1005B000AD0180E00E94981DFF91EF91BF91AF9136
:1005C0009F918F917F916F915F914F913F912F916B
:1005D0000F900BBE0F900FBE0F901F901895CF93EA
:1005E000DF931F92CDB7DEB7898321E0AE014F5F65
:1005F0005F4F60E080E00E94A50E8093AC010F90F9
:10060000DF91CF91089580B382FB882780F9089508
:1006100080916A00806180936A0080916A008F7D7A
:1006200080936A0089B7846089BF60E080E00E949F
:10063000861D0E940303811105C061E00E94861D92
:1006400080E005C062E080E00E94861D81E00C949D
:10065000EF02CF938091AD018F5F8093AD01873022
:10066000D0F10E940303C82F80E00E94A21D8111D7
:1006700004C08091AC01882361F180910601C81704
:1006800031F180E0C11111C00E948F1D682F6D7F74
:1006900080E00E94861D80E00E948F1D682F6160AF
:1006A00080E00E94861D80E010C00E948F1D682F90
:1006B0006E7F80E00E94861D80E00E948F1D682F63
:1006C000626080E00E94861D81E00E94EF02C0937C
:1006D00006011092AC01CF9108950C94C500809151
:1006E0008902882329F0109289020E94CE00FFCF50
:1006F0000895CF93DF93982FEB01FA01D90181334D
:1007000009F451C028F48E32B1F08F3211F168C073
:10071000833309F463C008F45FC0843309F060C018
:1007200080918A02808380918702818380918802F0
:10073000828383E00CC0108288E2818388E1828317
:10074000138214828CE0858381E0868387E08C931A
:100750003FC0898181113EC09A819230A1F060F43E
:10076000992369F09130E1F590839183128213828D
:100770001482158296E015C0953070F131C094E274
:10078000908391E00EC0C3E9D1E090E0983018F476
:100790002881208301C010829F5F219631969C3072
:1007A000A9F79C931EC08981811118C0809187028E
:1007B0008038B9F08A81813059F0823089F481E043
:1007C0008093890280E88093870290938A0209C00F
:1007D00080E007C082E805C083E803C081E801C06B
:1007E0008CECDF91CF910895D098D298D39AD49A77
:1007F000D59AB89ABB98BA98B998BD9ABE9ABF9A3A
:10080000A29AA39AA498A598A69AA79A8A981298A9
:100810001398E1E6F0E080818E7F8083E4E6F0E0EB
:100820008081816080838081826080838081846018
:1008300080838081877F8083089581E08093AF01EA
:100840000895AF9AAE9A80E00E948F1D682F677E50
:1008500080E00E94861D80E00895AF98AE9880E009
:100860000E948F1D682F606180E00E94861D80E0DD
:1008700008950E94D20B9091AE01882399F19111B5
:1008800013C080E00E941A05833870F080E00E9457
:100890008F1D682F6B7F80E00E94861D81E0809312
:1008A000AE010E9421040BC08091AE01813039F469
:1008B00080E00E941A05813410F41092AE018091FC
:1008C000AF011092AF01882371F10E942D0480E0E6
:1008D0000E948F1D682F646080E00E94861D82E068
:1008E0000C94EF0291110EC080E00E941A0583382B
:1008F00048F00E940303811105C081E08093AE019E
:100900000C9421048091AE01813069F480E00E9452
:100910001A05803420F41092AE010C942D040E942C
:1009200003038130C1F30895823059F4AF98AE9833
:10093000A89584EF91E00E94F21DAF9AAE9A80E0F4
:1009400008958FEF089584E008950F931F93CF9338
:10095000DF931F92CDB7DEB78E010F5F1F4F21E0EF
:1009600040E060E070E00E94CD0A89810F90DF9145
:10097000CF911F910F9108950F931F93CF93DF9302
:100980001F92CDB7DEB769838E010F5F1F4F21E045
:1009900040E060E070E00E94350A0F90DF91CF9157
:1009A0001F910F910895CF93DF93D82FC62F0E94E8
:1009B000A504C15061E070E001C0660FCA95EAF776
:1009C000609568238D2FDF91CF910C94BC04CF9359
:1009D000DF93D82FC62F0E94A504C15061E070E0BC
:1009E00001C0660FCA95EAF7682B8D2FDF91CF9172
:1009F0000C94BC0496B1987F892B86B9089527B1D1
:100A00002F7330E4839FC0011124822B87B908958E
:100A1000379A85E00E94FA0480E00E94FF043D9A24
:100A2000089597B1907E8F71892B87B90895349A74
:100A3000369A08950E9411050E941705349BFECF37
:100A400085B10895CF93DF9385E090E00E94BB00CD
:100A500028E0829FC00111240097D1F0EC01CE0163
:100A600001960E94BB009E012E5F3F4F87FD08C08C
:100A7000C9010E94BB0090E00596C80FD91FEFCFB7
:100A8000C9010E94BB0090E005968C0F9D1F22C0FB
:100A900084E090E00E94BB0038E0839FE0011124D5
:100AA000209751F483E090E00E94BB0098E0899F7A
:100AB000E0011124209761F0CE0101960E94BB0055
:100AC0009E0148E0849F200D311D1124C90102C000
:100AD00080E090E0DF91CF910895CF93DF93811173
:100AE00008C0EB010E942205888399831A8283E063
:100AF00001C08FEFDF91CF910895CF92DF92EF92F7
:100B0000FF920F931F93CF934D33F8F4F901C42F45
:100B1000DB01ED90FC904083811107C089010F5FDC
:100B20001F4F6701C40ED11C03C081E08C0F0EC0A3
:100B3000EC14FD04D1F3C7010E94BB00F8018193BE
:100B40008F01FFEFEF1AFF0AF3CF8FEFCF911F91C5
:100B50000F91FF90EF90DF90CF900895CF92DF92AA
:100B6000EF92FF920F931F93CF93DF93FC01C0800E
:100B7000D180842F90E09C012C0D3D1D2130384008
:100B8000B8F4C42FDFB7F8948B017B01E80EF91E8F
:100B90000E151F0551F0F80161918F01C6010E94E9
:100BA000B000FFEFCF1ADF0AF3CFDFBF8C2F01C0F9
:100BB0008FEFDF91CF911F910F91FF90EF90DF901A
:100BC000CF9008959F92AF92BF92CF92DF92EF9213
:100BD000FF920F931F93CF93DF93F82E8B0185E045
:100BE00090E00E94BB0028E0829FC0011124009782
:100BF00011F480E061C0EC01CE0101960E94BB00BF
:100C0000AE01485F5F4F6A0187FF06C0C6010E94C0
:100C1000BB00893171F70EC0CA010E94BB00893147
:100C2000A9F3CE0102960E94BB0090E00596C80F82
:100C3000D91FE2CFCE010A960E94BB0050E1859FEA
:100C4000C00DD11D1124CE010C960E94BB00F816D8
:100C500080F6CF2CD12C65E0F69E90011124F9018D
:100C600043E0849FE00DF11D1124CE0FDF1FCE0164
:100C70000D960E94BB00982ECE010E960E94BB00DE
:100C8000A82ECE010F960E94BB00B82ECE01409632
:100C90000E94BB00E82ECE0141960E94BB00F910D5
:100CA000A8CFF801A082B182E282F601EC54FE4F97
:100CB0008081F801838384E0DF91CF911F910F91B0
:100CC000FF90EF90DF90CF90BF90AF909F900895EE
:100CD000CF93DF93C82FD62F613019F40E94951E51
:100CE00004C0611109C00E94971E811105C0EC2F3C
:100CF000F0E0EC54FE4FD08380E0DF91CF91089577
:100D000080E00895FC0184E180831182128283E0F7
:100D10000895982F827091FF06C066956170609368
:100D2000B20180E0089590FF04C061706093B30148
:100D300008958FEF08958091B201880F827090918D
:100D4000B301892B80938B020895813031F4809117
:100D5000B1018F5F8093B10107C08091B001811113
:100D600003C081E08093B00180E0089580E090E0CE
:100D70000E94BB008F3F11F40C9455020895BC01F2
:100D8000809171008E7F80937100809171008D7FC2
:100D90008093710080E991E00E949B1E862F603154
:100DA00038F07727CB01409797FD01969595879569
:100DB000809370000895909A919A1092C8011092B1
:100DC000C70184E190E00E94BF06E4E7F0E0808183
:100DD000846080831092630280818160808380813F
:100DE0008064808308958E7F91E0611101C090E05E
:100DF000982B9093720008959093C8018093C70137
:100E00000895E4E7F0E080818F70806A8083089520
:100E1000E4E7F0E080818F70806D80830895809397
:100E20007300E4E7F0E080818F708068808308952C
:100E3000882329F0809174008F70806C04C08091A9
:100E400074008F708068809374000895909163029D
:100E50009111FCCF92E0909363028E7F80936202A7
:100E6000942FA7E1B2E0FA018E2F891B861718F4A0
:100E700081918D93F9CF10921602609315020C9414
:100E800001071F920F920FB60F9211240BB60F920B
:100E90002F933F934F935F936F937F938F939F9382
:100EA000AF93BF93EF93FF9380917100887F80375A
:100EB00009F467C020F5803209F44AC080F4883014
:100EC00009F443C038F48111BDC0809174008F7063
:100ED000806DB4C08031C9F18831D1F1B3C088339D
:100EE00009F44AC028F4883299F1803389F1AAC004
:100EF000803609F446C0883609F443C0A3C0803A5E
:100F000009F45CC080F4883809F454C030F48837A0
:100F1000C1F1803809F440C095C08039E9F18839C1
:100F200009F448C08FC0883B09F466C038F4883A99
:100F300009F456C0803B09F453C084C0803C09F4D6
:100F400079C0883C09F476C07DC0809162020EC0F1
:100F5000E091160280911502E81758F481E08E0F97
:100F600080931602F0E0E95EFD4F80810E940F073A
:100F700069C00E94080764C0809174008F70806807
:100F80005DC085E08093630281E08093C901809118
:100F900073008093CA0142C0E091C90181E08E0FC5
:100FA0008093C90190917300F0E0E653FE4F908367
:100FB0008032A0F180E00E94180744C08091740044
:100FC0008F70806C80937400E091C701F091C8012C
:100FD0003097B1F16AEC71E08091C901099530C098
:100FE00084E080936302E091C501F091C6016AEC50
:100FF00071E08091C9010995E091160281E08E0FA0
:1010000080931602F0E0E95EFD4F808180937300CB
:101010009091160280911502981728F4809174001F
:101020008F70806C04C0809174008F708068809392
:10103000740008C0809174008F70806C809374007D
:1010400010926302FF91EF91BF91AF919F918F91A9
:101050007F916F915F914F913F912F910F900BBEB8
:101060000F900FBE0F901F90189527E030E090E092
:10107000AC01022E02C0559547950A94E2F740FF55
:1010800002C08D9801C08D9A000000000000000091
:101090000000000000000000000000000000000050
:1010A0000000000000000000000000000000000040
:1010B0000000000000000000000000000000000030
:1010C0000000000000000000000000000000000020
:1010D00000000000000000008C98000000000000EC
:1010E0000000000000000000000000000000000000
:1010F00000000000000000000000000000000000F0
:1011000000000000000000000000000000000000DF
:1011100000000000000000000000000000000000CF
:10112000000000000000000000008C9A21503109EE
:1011300008F09ECF8D980000000000000000000025
:10114000000000000000000000000000000000009F
:10115000000000000000000000000000000000008F
:10116000000000000000000000000000000000007F
:10117000000000000000000000000000000000006F
:101180000000000000008C9880B300000000000008
:10119000000000000000000000000000000000004F
:1011A000000000000000000000000000000000003F
:1011B000000000000000000000000000000000002F
:1011C000000000000000000000000000000000001F
:1011D000000000000000000000008C9A00000000E9
:1011E00000000000000000000000000000000000FF
:1011F00000000000000000000000000000000000EF
:1012000000000000000000000000000000000000DE
:1012100000000000000000000000000000000000CE
:1012200000000000000000000000000085FB88278F
:1012300080F991E089270895AC018D9828E030E08D
:1012400080E000000000000000000000000000003E
:10125000000000000000000000000000000000008E
:10126000000000000000000000000000000000007E
:10127000000000000000000000000000000000006E
:10128000000000000000000000000000000000005E
:1012900000008C98880F8599816000000000000094
:1012A000000000000000000000000000000000003E
:1012B000000000000000000000000000000000002E
:1012C000000000000000000000000000000000001E
:1012D000000000000000000000000000000000000E
:1012E000000000000000000000008C9A215031092D
:1012F00009F0A7CF8D9A452B11F08D9801C08D9ADA
:1013000000000000000000000000000000000000DD
:1013100000000000000000000000000000000000CD
:1013200000000000000000000000000000000000BD
:1013300000000000000000000000000000000000AD
:10134000000000000000000000000000000000009D
:101350008C98000000000000000000000000000069
:10136000000000000000000000000000000000007D
:10137000000000000000000000000000000000006D
:10138000000000000000000000000000000000005D
:10139000000000000000000000000000000000004D
:1013A00000008C9A8D980895959894988D988C98B3
:1013B000000000000000000000000000000000002D
:1013C000000000000000000000000000000000001D
:1013D000000000000000000000000000000000000D
:1013E00000000000000000000000000000000000FD
:1013F00000000000000000000000000000000000ED
:101400008C980000000000000000000000000000B8
:101410000000000000008D980000000000000000A7
:1014200000000000000000000000000000000000BC
:1014300000000000000000000000000000000000AC
:10144000000000000000000000000000000000009C
:10145000000000000000000000000000000000008C
:1014600000000000000000000895DF92EF92FF925C
:101470000F931F93CF93DF93F62EE72ED42FC22F17
:10148000DFB6F8948D9A0000000000000000000014
:10149000000000000000000000008C9A880F0E94ED
:1014A0003508D23041F48E2D0E9435088F2D0E94D0
:1014B0003508780103C0D130E1F7F8CFCC2339F0FB
:1014C000F70181917F010E943508C150F7CF8D9AB5
:1014D000000000000000000000000000000000000C
:1014E00000000000000000000000000000000000FC
:1014F00000000000000000000000000000000000EC
:1015000000000000000000000000000000000000DB
:1015100000000000000000000000000000000000CB
:101520008C98000000000000000000000000000097
:101530000000000000008D98000000000000000086
:10154000000000000000000000000000000000009B
:10155000000000000000000000000000000000008B
:10156000000000000000000000000000000000007B
:10157000000000000000000000000000000000006B
:101580000000000000000000DFBEDF91CF911F913E
:101590000F91FF90EF90DF900895AF92BF92DF928E
:1015A000EF92FF920F931F93CF93DF93E62EB72E08
:1015B000F42EC22FD82FDD0FDFB6F8948D9A0000DD
:1015C000000000000000000000000000000000001B
:1015D00000008C9A82E0481305C08D2F0E943508C8
:1015E0008B2D04C0E1E04E1306C08D2F0E943508FC
:1015F0008E2D0E9435080000000000000000000051
:1016000000000000000000000000000000000000DA
:1016100000000000000000000000000000000000CA
:1016200000000000000000000000000000000000BA
:1016300000000000000000000000000000000000AA
:10164000000000000000FF2069F08C988D9A0000D7
:10165000000000000000000000000000000000008A
:1016600000008C9A8D2F81600E94350878010C2F24
:1016700010E0C0E0D0E05801F1E0AF1AB1080C175B
:101680001D0771F081E090E0AC16BD0611F080E01E
:1016900090E00E941C09F70181937F012196EFCF12
:1016A0008D9A000000000000000000000000000013
:1016B000000000000000000000000000000000002A
:1016C000000000000000000000000000000000001A
:1016D000000000000000000000000000000000000A
:1016E00000000000000000000000000000000000FA
:1016F00000008C98000000000000000000000000C6
:1017000000000000000000008D98000000000000B4
:1017100000000000000000000000000000000000C9
:1017200000000000000000000000000000000000B9
:1017300000000000000000000000000000000000A9
:101740000000000000000000000000000000000099
:1017500000000000000000000000DFBEDF91CF911C
:101760001F910F91FF90EF90DF90BF90AF90089581
:101770009091840598609093840590FD12C0262F67
:10178000A8ECB5E0FB019E2F921B981718F49191DD
:101790009D93F9CF80931306809184058160809397
:1017A000840508958091640208958093BA06609339
:1017B000B9068F3F19F410926502089581E0809375
:1017C00065020895E5E8F5E0108280E8818381E014
:1017D0008283838381E5848389E2858380E68683AF
:1017E0001782108681E4818787E582878BE00895E0
:1017F0000F931F93CF93DF93CDB7DEB7CC54D109AE
:101800000FB6F894DEBF0FBECDBF082F8091C6057E
:1018100089838091BB0690E00196880F991F880FFD
:10182000991F9091BC069370892B8A8362E0CE0148
:1018300001960E947F1E8B83809168068C83809125
:101840000107880F880F8D838091BD068E830F83DB
:101850008091BB068C3219F4188618E001C017E09D
:10186000011113C080916706882379F0E5E8F5E05F
:10187000810F181751F09191A1E0B0E0AC0FBD1F9E
:10188000A10FB11D9C931F5FF4CF612FCE01019674
:101890000E947F1EE1E0F0E0EC0FFD1FE10FF11D63
:1018A0008083AE014E5F5F4F612F8091C6050E941D
:1018B0002607809184058E7F80938405C45BDF4F6B
:1018C0000FB6F894DEBF0FBECDBFDF91CF911F9151
:1018D0000F910895AF92CF92EF920F9310926706F7
:1018E00020916602422F50E09091BB06FA01EA5E19
:1018F000F94F90838091BD06FA01E759F94F808333
:101900002F5F2F3418F42093660202C010926602F3
:101910009A3009F4ACC028F4943099F0963059F01C
:101920006DC19E3209F4E9C0903309F4E6C09C32DF
:1019300009F4D2C063C1813009F060C10E94E20B9A
:10194000DAC0813281F160F4813031F1F0F080321F
:1019500009F054C160E085E895E00E94CF1BCBC040
:10196000863209F45BC020F4823209F46AC046C1B1
:10197000873209F446C08D3209F040C165E875E050
:101980008091C0060E94461D42C06091C1068091B0
:10199000C0060E94D50BB1C08091BA068093850520
:1019A0008091B90660C06091C406662321F18091E0
:1019B0006702909168022091C00630E0AC01552783
:1019C0002417350709F018C12091C10630E0892F8E
:1019D00099272817390709F00FC125E835E040910C
:1019E000C50682EC96E00E94DA1B809367068F3F63
:1019F00009F083C005C125E835E04091C50660E0E7
:101A0000F0CF65E875E08091C0060E94261C8093A7
:101A100067068F3F09F071C08DECF3C0A090C70638
:101A2000C090C606E090C5060091C4062091C3068A
:101A30004091C2066091C1068091C0060E94A81C18
:101A4000E6CF8091670290916802019611F481E0DF
:101A500090E0909368028093670290916702809172
:101A60006802909385058093860582E044C08131A9
:101A700081F08231C9F0803109F0C0C065E875E0BD
:101A80008091C0060E946D05809367068F3FA9F57F
:101A9000B5C025E835E04091C30661EC76E0809161
:101AA000C0060E947D05A1CF8091C00681110DC0A6
:101AB0004091BE06435063EC76E081EC96E00E94D4
:101AC000AE058093670680E001C081EC90916706C7
:101AD0009F3F09F096C094C0482F50E04D32510509
:101AE00008F081C0FA01EA5BFF4F0C94AF1E85E855
:101AF00095E00E9482068093670680E082C081E0C4
:101B0000809367060E94A30480938505F6CF909189
:101B1000C1068091C206913019F4843009F46EC078
:101B2000843019F40E941D04E8CF0E9494048F3F72
:101B300021F78CEC66C065E875E08091C1060E94D3
:101B40003210D9CF45E855E06091C2068091C106B8
:101B50000E943D100AC02091C4064091C3066091C6
:101B6000C2068091C1060E94821380936706DFCF70
:101B700045E855E06091C2068091C1060E94FB0FC6
:101B8000F4CF8091C2060E94A506D1CF6091C30612
:101B90008091C2060E948906CACF0E949B0680934C
:101BA000850581E0A8CF8091C206811129C065E832
:101BB00075E08091C1060E94791D17CF6091C5061E
:101BC0008091C1060E94680696CF65E875E0809115
:101BD000C1060E94E2058FCF6091C3068091C106C5
:101BE0000E94800688CF27E636E045E855E060ECA5
:101BF00076E00E94790305C085EC03C081EC01C04A
:101C000089EC0F91EF90CF90AF900C94F80B8091EE
:101C1000840580FF99C04091CA0562E088EC95E098
:101C20000E948C1E811190C060911306E62FF0E097
:101C3000E953FA4F6150408188EC95E00E948C1E78
:101C4000811182C08091C805809368068091C90582
:101C5000869586958093BB062091CB052093C6057B
:101C60009091CC05392F36953695309301079370B6
:101C70009093BC069091CD059093BD0680FF3FC028
:101C80008091BA06281360C0809184058E7F80936E
:101C9000840510926606109202078091CE05882373
:101CA00021F080916902833030F181E02CE4909141
:101CB0006A028917D0F4482F50E0BA0161507109C7
:101CC000269FD001279FB00D1124A457BD4F249FFC
:101CD000F001259FF00D1124E457FD4F922F019044
:101CE0000D929A95E1F78F5FE2CF915090936A023F
:101CF0001092690208958F5F809369020895809120
:101D000013068830D8F090E09C01275031093093B9
:101D1000BF062093BE0646E00197EAEFE40F242FAA
:101D200030E02817390774F4F0E0E554F94FD90191
:101D3000A853BA4F2C9125834F5FEFCF1092BF0667
:101D40001092BE060C946A0C0895CF92DF92EF9227
:101D5000FF920F931F93CF93DF93C0916A02CA3013
:101D600008F05EC0022F7A01D62EC82E909115067B
:101D70009F5F909315061CE41C9FE0011124C4573B
:101D8000DD4F990F990F9C8382E08D8384E08E83D1
:101D90008C2D0E94AC1D8F83C0916A021C9FE001B4
:101DA0001124C457DD4FC8868C2D0E94B51D8F7736
:101DB000D82AD98680916A02282F30E0002319F0B2
:101DC000F701908101C09FEF4CE4429FF001439FD7
:101DD000F00D1124E457FD4F9287023018F0F701FF
:101DE000918101C09FEF4CE4429FF001439FF00DB1
:101DF0001124E457FD4F9387033018F0F7019281C7
:101E000001C09FEF4CE4429FF001439FF00D11246D
:101E1000E457FD4F94878F5F80936A0280E001C092
:101E200081E0DF91CF911F910F91FF90EF90DF90B4
:101E3000CF900895CF93DF9381E080930207CCE8A1
:101E4000D2E08091BA0688838091B9068370806160
:101E50008983809114068B8362E0CE010E947F1EED
:101E60008A836DE0CE010E947F1E8D874DE852E08F
:101E70006DE08091BA06DF91CF910C942607809196
:101E8000BA068F3F69F080916A02882349F08091F9
:101E90000207811105C08091840580FF0C941A0F00
:101EA00008951F93CF93DF93BB98BA98B998B89AC7
:101EB000C09880B5846080BD84E690E00E94DE1DFD
:101EC00026B323FB112710F996B392FBDD27D0F937
:101ED00086B381FBCC27C0F9C09A84E690E00E94CB
:101EE000DE1D86B383FB882780F9181302C0212FDB
:101EF00001C022E086B382FB882780F9D81302C094
:101F00009D2F01C092E086B386958170C81302C0F0
:101F10008C2F01C082E021110EC0911104C08230CB
:101F2000F1F582E73DC09230D1F5882361F182302E
:101F3000B1F586E735C02230B1F4911106C088238F
:101F400021F1823061F58AE72BC0923031F4882389
:101F5000F1F0813021F58EE723C08230D1F081305D
:101F6000F1F482E81DC0923031F48230A1F081306A
:101F7000B1F486E815C0913091F4823071F081306F
:101F800071F484EA0DC084E70BC088E709C08CE7D0
:101F900007C080E805C084E803C088E801C080E08D
:101FA00090B59B7F90BD811101C080E7DF91CF91FB
:101FB0001F9108950E94DB060E94510F8093140622
:101FC0006FEF0E94F30688EB9BE00E94FC068FEF08
:101FD0008093BA0681E0809315061092B90610929C
:101FE000660680936402089580911406811102C0F0
:101FF0000C94510F0895DA0181112EC0633060F501
:102000008CE0689FF0011124ED5FF84F84818C9380
:10201000808111968C931197828112968C931297DE
:10202000838113968C93139784818B7F8230B1F4D4
:10203000818114968C931497828115968C931597B1
:10204000838116968C9316978481863049F4868115
:1020500017968C9388E008958FEF089584E0089593
:1020600087E00895FB0197E09083811103C083E02E
:10207000818301C0118282E00895DA0181111AC0C2
:102080006330C0F48CE0689FF0011124ED5FF84FDD
:1020900081E090E0038002C0880F991F0A94E2F764
:1020A0008C93838111968C931197838112968C93D4
:1020B00083E008958FEF0895DC0116968C911697B2
:1020C0001296EC9112974E2F50E0882309F461C0CC
:1020D0004730510508F0CDC0FA01ED58FF4F139677
:1020E0008C910C94AF1E4BB321E030E0B90102C0DB
:1020F000660F771F8A95E2F7CB01842B61C048B346
:1021000021E030E0B90102C0660F771F8A95E2F73F
:10211000CB01842B63C045B321E030E0B90102C09C
:10212000660F771F8A95E2F7CB01842B65C042B317
:1021300021E030E0B90102C0660F771F8A95E2F70F
:10214000CB01842B67C043B121E030E0B90102C06C
:10215000660F771F8A95E2F7CB01842B69C0409107
:10216000620021E030E0B90102C0660F771F8A9556
:10217000E2F7CB01842B6BC04091650021E030E099
:10218000B90102C0660F771F8A95E2F7CB01842B55
:102190006EC04730510508F06CC0FA01E658FF4F99
:1021A00013968C910C94AF1E4BB321E030E0B90133
:1021B00002C0660F771F8A95E2F7CB0180958423D2
:1021C0008BBB089548B321E030E0B90102C0660F2F
:1021D000771F8A95E2F7CB018095842388BB089509
:1021E00045B321E030E0B90102C0660F771F8A9540
:1021F000E2F7CB018095842385BB089542B321E0AB
:1022000030E0B90102C0660F771F8A95E2F7CB0173
:102210008095842382BB089543B121E030E0B90169
:1022200002C0660F771F8A95E2F7CB018095842361
:1022300083B908954091620021E030E0B90102C005
:10224000660F771F8A95E2F7CB01809584238093F0
:10225000620008954091650021E030E0B90102C0BC
:10226000660F771F8A95E2F7CB01809584238093D0
:1022700065000895DC0117968C9117971296EC91E2
:1022800012974E2F50E0882309F461C04730510562
:1022900008F0CDC0FA01EF57FF4F13968C910C94C4
:1022A000AF1E4BB321E030E0B90102C0660F771FCB
:1022B0008A95E2F7CB01842B61C048B321E030E07E
:1022C000B90102C0660F771F8A95E2F7CB01842B14
:1022D00063C045B321E030E0B90102C0660F771F4B
:1022E0008A95E2F7CB01842B65C042B321E030E050
:1022F000B90102C0660F771F8A95E2F7CB01842BE4
:1023000067C043B121E030E0B90102C0660F771F1A
:102310008A95E2F7CB01842B69C04091620021E0ED
:1023200030E0B90102C0660F771F8A95E2F7CB0152
:10233000842B6BC04091650021E030E0B90102C000
:10234000660F771F8A95E2F7CB01842B6EC047306A
:10235000510508F06CC0FA01E857FF4F13968C91B5
:102360000C94AF1E4BB321E030E0B90102C0660F00
:10237000771F8A95E2F7CB01809584238BBB089564
:1023800048B321E030E0B90102C0660F771F8A959B
:10239000E2F7CB018095842388BB089545B321E003
:1023A00030E0B90102C0660F771F8A95E2F7CB01D2
:1023B0008095842385BB089542B321E030E0B901C4
:1023C00002C0660F771F8A95E2F7CB0180958423C0
:1023D00082BB089543B121E030E0B90102C0660F2D
:1023E000771F8A95E2F7CB018095842383B90895FE
:1023F0004091620021E030E0B90102C0660F771F12
:102400008A95E2F7CB01809584238093620008953A
:102410004091650021E030E0B90102C0660F771FEE
:102420008A95E2F7CB018095842380936500089517
:10243000EF92FF921F93CF93DF93CDB7DEB7E09774
:102440000FB6F894DEBF0FBECDBF28E1FE0179962E
:10245000DF01922F1D929A95E9F791E09B8F37E06B
:102460003C8F9D8F98A39BA335E03CA332E03DA316
:102470003FEF3EA398A79BA736E03CA733E03DA7DC
:1024800098ABDE01119601900D922A95E1F7E62EA8
:10249000F12CACE06A9FF0011124ED5FF84F9481BC
:1024A0009B7F9230E1F1142F81112FC0F70183E05F
:1024B000EE0FFF1F8A95E1F781E090E08C0F9D1FE2
:1024C000E80FF91F8081882319F0813069F01DC061
:1024D0004F3F21F4CF010E945C1017C0411115C07D
:1024E000CF010E943A1111C04F3F11F4868103C001
:1024F00041110BC087816381882321F081810E9473
:10250000E70403C081810E94D3048CE08E9DF0011A
:102510008F9DF00D1124ED5FF84F10831583E09629
:102520000FB6F894DEBF0FBECDBFDF91CF911F91E4
:10253000FF90EF900895CF92DF92EF92FF920F936A
:102540001F93CF93DF93CDB7DEB7E0970FB6F89424
:10255000DEBF0FBECDBF98E1FE017996DF01892F66
:102560001D928A95E9F781E08B8F27E02C8F8D8F64
:1025700088A38BA325E02CA322E02DA32FEF2EA36D
:1025800088A78BA726E02CA723E02DA788ABDE0128
:10259000119601900D929A95E1F7DE0111967D0159
:1025A00003E017E0D12CCC24C394F7014581D80176
:1025B0004C9311964C93119712961C92129784810A
:1025C00013968C9313971496CC926D2D80E00E94F5
:1025D0001812D394B8E0EB0EF11C045F1F4FE3E038
:1025E000DE12E3CFE0960FB6F894DEBF0FBECDBF8C
:1025F000DF91CF911F910F91FF90EF90DF90CF90DF
:102600000895EF92FF921F93CF93DF93CDB7DEB77C
:10261000E0970FB6F894DEBF0FBECDBF28E1FE01F4
:102620007996DF01922F1D929A95E9F791E09B8FA1
:1026300037E03C8F9D8F98A39BA335E03CA332E00D
:102640003DA33FEF3EA398A79BA736E03CA733E00E
:102650003DA798ABDE01119601900D922A95E1F706
:10266000E62EF12CACE06A9FF0011124ED5FF84FEB
:1026700094819130D9F1142F81112FC0F70183E09B
:10268000EE0FFF1F8A95E1F781E090E08C0F9D1F10
:10269000E80FF91F8081882319F0813069F01DC08F
:1026A0004F3F21F4CF010E945C1017C0411115C0AB
:1026B000CF010E943A1111C04F3F11F4868103C02F
:1026C00041110BC087816381882321F081810E94A1
:1026D000E70403C081810E94D3048CE08E9DF00149
:1026E0008F9DF00D1124ED5FF84F1583E0960FB626
:1026F000F894DEBF0FBECDBFDF91CF911F91FF9049
:10270000EF900895811145C0633008F042C0A62FB4
:10271000B0E08CE0689FF0011124ED5FF84F8481F8
:102720008630B9F19FEF940F9A3F30F441832283B2
:1027300082E08483238727C09E3F28F04183128252
:1027400082E0848321C04C3F39F481E0848340815E
:1027500080E00E9418121BC04B3FD9F427FD19C01E
:10276000813011F48CEF01C0818187838CE08A9FD6
:10277000F0018B9FF00D1124ED5FF84F86E084830C
:102780002683118610864FEF80E00E94011380E0BF
:1027900008958FEF08951F93CF93DF93C3E0D7E0A1
:1027A00010E08C818630A9F48885998501969987F7
:1027B00088872E814AE0249F900111248217930775
:1027C00008F11C822A814F81612F80E00E948213D0
:1027D00019C099818FEF890F8A3FA0F48B858250B1
:1027E0008B8781110FC08D81882329F08F3F51F491
:1027F0009B8740E003C08A818B874FEF612F80E089
:102800000E9401132C961F5F133059F6DF91CF9170
:102810001F9108950E946D030E94F4030E94B60662
:102820000E94D4090E949B120E9408050E946D1408
:102830000E94F0140E94BE1D88B1479A0E94941E07
:102840000E94DA0F0E94101E0E94080340E061E01F
:1028500080E00E941812789480E008950FB6F894F2
:10286000A89581B5886181BD11BC0FBE0E940A1474
:10287000811130C09FE088E10FB6F894A89581BD22
:102880000FBE91BDA8950E94070E0E9439040E94B8
:102890006F030E94290380E00E941A05813810F01E
:1028A0004FEF01C040E062E080E00E9418120E94F9
:1028B0007A1E882321F00E94BE1D0E943F0F85B71B
:1028C000837E85BF85B7806285BF889585B78F7DFC
:1028D00085BFD8CF80E090E00895CF93DF930E942A
:1028E000F40F91E0909327071092280791E59093B9
:1028F000290792E190932A0796E190932B07109273
:102900002C0710922D0710922E0799E290932F0713
:1029100010923007109231071092320791EC909389
:10292000330710923407109235079EEC90933607C8
:10293000ECE9F1E0A7E3B7E091919D9391E0EA3AE9
:10294000F907D1F723E431E03093800720937F0724
:1029500093E39093830727E031E030937E07209341
:102960007D079CE39093820727E237E030937C0752
:1029700020937B079EE190938107282F30E020571A
:102980003109359527952066C1E8D7E0EBE7F7E0F8
:1029900090E0A081B1813991355014963C93A0818B
:1029A000B18113963C9113974FEF430F423020F4BF
:1029B00019962C93199705C0323119F41D962C9352
:1029C0001D979C93A081B18111961C92A191B19108
:1029D00015968C939F5F9330E1F6DF91CF91089528
:1029E000CF93DF93E5E4F7E020E030E060ECABE785
:1029F000B7E080E0CD91DD919B819150923038F429
:102A00004F81042E000C550B4217530719F08F5FAE
:102A1000833081F7A82FB0E0AA0FBB1FA558B84F8D
:102A20000D90BC91A02D13969C91139790831C96AA
:102A30009C911C9795831D969C911D97978311825D
:102A40001382148212828087668313968C91139767
:102A5000813009F045C054968C915497807C91E068
:102A600009F490E091871E968D919C911F9798276D
:102A700089279827968B858B50968D919C9151979D
:102A8000982789279827908F878B5F968C915F97DF
:102A9000828790968C919097838791968C9191974D
:102AA000848794968C919497858795968C91959729
:102AB000868796968C919697878797968C9197970D
:102AC000808B98968C919897818B99968C919997F9
:102AD000828B9A968C919A97838B9B968C91848B00
:102AE0002F5F3F4F7B962230310509F080CFDF9179
:102AF000CF910C94991ECF92DF92EF92FF920F9399
:102B00001F93CF93DF931F92CDB7DEB7C82ED12C82
:102B10009BE1899F9001112489010B5B184FF801FB
:102B2000E080F1E0EF1231C6F82EF80183818430A5
:102B300009F446C548F4813009F43CC308F405C3E0
:102B4000823009F42FC417C6803109F4DEC0803208
:102B500021F0883009F00FC6DFC1F801918561814D
:102B600085854389992309F466C0062E000C770BEE
:102B7000082E000C990B042E000C550B4F5F5F4F75
:102B8000841B950B86179707E4F0F901E25AF84F7A
:102B9000808180FF0CC09BE099838E7F808321E041
:102BA000AE014F5F5F4F60E88C2D0E94A50E8BE158
:102BB0008C9DF0018D9DF00D1124EB5BF84F80E1B1
:102BC00083838BE18C9DF0018D9DF00D1124DF013D
:102BD000AB5BB84F14969C91149713968C911397F6
:102BE000981761F011969C9111971D968C918917F9
:102BF0002CF0E25AF84F808181FF60C08BE18C9D00
:102C0000F0018D9DF00D1124DF01AB5BB84F1196E3
:102C10002C911197022E000C330B54968C915497E3
:102C2000082E000C990B01961D964C91840F911D56
:102C300047FD9A955DC070E090E050E04F5F5F4FB8
:102C4000841B950B86179707E4F0F901E25AF84FB9
:102C5000808180FF0CC09BE099838E7F808321E080
:102C6000AE014F5F5F4F60E88C2D0E94A50E8BE197
:102C70008C9DF0018D9DF00D1124EB5BF84F80E1F0
:102C800083838BE18C9DF0018D9DF00D1124DF017C
:102C9000AB5BB84F14969C91149713968C91139735
:102CA000981781F011969C9111971D968C91891718
:102CB00048F0E25AF84F808181FD04C09AE0998380
:102CC000826026C58BE18C9DF0018D9DF00D112455
:102CD000DF01AB5BB84F11962C91119730E0549601
:102CE0008C91549790E001961D964C91840F911D04
:102CF000281739070CF43FC5E25AF84F808181FF4D
:102D00003AC59AE099838D7F2DC5F801418581816F
:102D10009585442309F47EC089179CF08BE0898354
:102D2000F901E25AF84F80818160808321E0AE0191
:102D30004F5F5F4F60E08C2D0E94A50E80E2F8018E
:102D40002EC0082E000C990BF8014685042E000CAD
:102D5000550B6389062E000C770B6F5F7F4F461B68
:102D6000570B48175907E4F0F901E25AF84F8081F0
:102D700082FF0CC099E099838B7F808321E0AE01B4
:102D80004F5F5F4F60E88C2D0E94A50E8BE18C9DFC
:102D9000F0018D9DF00D1124EB5BF84F88E08383EB
:102DA0008BE18C9DF0018D9DF00D1124DF01AB5B5B
:102DB000B84F14969C91149713968C91139798176B
:102DC00061F011969C9111971E968C9189172CF0A9
:102DD000E25AF84F808183FF78C08BE18C9DF0012F
:102DE0008D9DF00D1124DF01AB5BB84F11962C9136
:102DF0001197022E000C330B54968C915497082E89
:102E0000000C990B01961E964C91840F911D47FD65
:102E10009A9575C0891798F08BE08983F901E25A79
:102E2000F84F80818160808321E0AE014F5F5F4F6A
:102E300060E08C2D0E94A50E80E2F80128C090E091
:102E4000F801468550E0638970E06F5F7F4F461B55
:102E5000570B48175907E4F0F901E25AF84F8081FF
:102E600082FF0CC099E099838B7F808321E0AE01C3
:102E70004F5F5F4F60E88C2D0E94A50E8BE18C9D0B
:102E8000F0018D9DF00D1124EB5BF84F88E08383FA
:102E90008BE18C9DF0018D9DF00D1124DF01AB5B6A
:102EA000B84F14969C91149713968C91139798177A
:102EB00081F011969C9111971E968C91891748F07C
:102EC000E25AF84F808183FD04C098E099838860BE
:102ED0001FC48BE18C9DF0018D9DF00D1124DF014D
:102EE000AB5BB84F11962C91119730E054968C91B2
:102EF000549790E001961E964C91840F911D2817CF
:102F000039070CF438C4E25AF84F808183FF33C488
:102F100098E09983877F26C4F80141858181968551
:102F2000442309F487C08917A4F089E08983F90153
:102F3000E25AF84F80818460808321E0AE014F5FC8
:102F40005F4F60E08C2D0E94A50E80E1F801838325
:102F500037C0082E000C990BF8014785042E000C91
:102F6000550B6389062E000C770B6F5F7F4F461B56
:102F7000570B4817590724F1F901E25AF84F80819D
:102F800084FF15C087E089838BE18C9DF0018D9DC6
:102F9000F00D1124E25AF84F80818F7E808321E06A
:102FA000AE014F5F5F4F60E88C2D0E94A50E8BE154
:102FB0008C9DF0018D9DF00D1124EB5BF84F138279
:102FC0008BE18C9DF0018D9DF00D1124DF01AB5B39
:102FD000B84F14969C91149713968C911397981749
:102FE00061F011969C9111971F968C9189172CF086
:102FF000E25AF84F808185FF81C08BE18C9DF00102
:103000008D9DF00D1124DF01AB5BB84F11962C9113
:103010001197022E000C330B54968C915497082E66
:10302000000C990B01961F964C91840F911D47FD42
:103030009A957EC08917A0F089E08983F901E25A48
:10304000F84F80818460808321E0AE014F5F5F4F45
:1030500060E08C2D0E94A50E80E1F801838331C0D1
:1030600090E0F801478550E0638970E06F5F7F4F23
:10307000461B570B4817590724F1F901E25AF84F3C
:10308000808184FF15C087E089838BE18C9DF001EE
:103090008D9DF00D1124E25AF84F80818F7E808340
:1030A00021E0AE014F5F5F4F60E88C2D0E94A50EBE
:1030B0008BE18C9DF0018D9DF00D1124EB5BF84FA1
:1030C00013828BE18C9DF0018D9DF00D1124DF01A9
:1030D000AB5BB84F14969C91149713968C911397F1
:1030E000981781F011969C9111971F968C918917D2
:1030F00048F0E25AF84F808185FD04C096E099833C
:10310000806206C38BE18C9DF0018D9DF00D112432
:10311000DF01AB5BB84F11962C91119730E05496BC
:103120008C91549790E001961F964C91840F911DBD
:10313000281739070CF41FC3E25AF84F808185FF26
:103140001AC396E099838F7D0DC3F8014185818173
:103150009785442341F0891744F4F8019289981720
:103160000CF409C31BC08917A0F087E08983F9011B
:10317000E25AF84F80818061808321E0AE014F5F89
:103180005F4F60E08F2D0E94A50E88E0F8018383D9
:10319000F2C2F8019289981708F4EDC2198221E071
:1031A000AE014F5F5F4F60E08F2D0E94A50EF801CA
:1031B000E382E1C2F801518541819189552309F4E7
:1031C00072C09417A4F083E08983F901E25AF84FA2
:1031D00081818160818321E0AE014F5F5F4F60E0BC
:1031E0008C2D0E94A50E82E0F80183832DC0042E51
:1031F000000C550BF8016389062E000C770B6F5FEE
:103200007F4F9289690F711D97FD7A954617570771
:10321000DCF0F901E25AF84F908194FF0CC08983E9
:1032200081818B7F818321E0AE014F5F5F4F60E83A
:103230008C2D0E94A50E8BE18C9DF0018D9DF00DD3
:103240001124EB5BF84F13828BE18C9DF0018D9D77
:10325000F00D1124DF01AB5BB84F14969C911497CD
:1032600013968C911397981741F011969C91119792
:1032700052968C9198170CF06BC02BE12C9DC001DD
:103280002D9D900D1124FC01EB5BF84F6181062E02
:10329000000C770B2289022E000C330B4489042E7C
:1032A000000C550B6AC09417A0F083E08983F901E4
:1032B000E25AF84F81818160818321E0AE014F5F46
:1032C0005F4F60E08C2D0E94A50E82E0F8018383A1
:1032D00027C050E0F801638970E06F5F7F4F9289EB
:1032E000690F711D46175707DCF0F901E25AF84FD4
:1032F000908194FF0CC0898381818B7F818321E041
:10330000AE014F5F5F4F60E88C2D0E94A50E8BE1F0
:103310008C9DF0018D9DF00D1124EB5BF84F138215
:103320008BE18C9DF0018D9DF00D1124DF01AB5BD5
:10333000B84F14969C91149713968C9113979817E5
:1033400069F011969C91119752968C91981730F0D4
:103350001982E25AF84F8181886020C12BE12C9DAF
:10336000C0012D9D900D1124FC01EB5BF84F618194
:1033700070E0228930E0448950E04F5F5F4F241BAA
:10338000350B261737070CF4F6C1FC01E15AF84F4C
:10339000208123FFF0C11982FC01E25AF84F81819C
:1033A000877F96C0F801418581819089442309F483
:1033B00091C098179CF085E08983F901E25AF84F93
:1033C00080818064808321E0AE014F5F5F4F60E0C9
:1033D0008C2D0E94A50E84E0F80136C0082E000C4A
:1033E000990BF8014389042E000C550B4F5F5F4F7A
:1033F0006189460F511D67FD5A95841795072CF179
:10340000F901E25AF84F808182FF15C083E0898379
:103410008BE18C9DF0018D9DF00D1124E25AF84F47
:1034200081818E7F818321E0AE014F5F5F4F60E835
:103430008C2D0E94A50E8BE18C9DF0018D9DF00DD1
:103440001124EB5BF84F81E083838BE18C9DF001CD
:103450008D9DF00D1124DF01AB5BB84F14969C914C
:10346000149713968C911397981741F011969C918D
:10347000119751968C9198170CF08AC02BE12C9DD6
:10348000C0012D9D900D1124FC01EB5BF84F618173
:10349000062E000C770B2189022E000C330B448979
:1034A000042E000C550B4F5F5F4F241B350B261766
:1034B00037070CF460C1FC01E15AF84F208121FF6D
:1034C0005AC122E02983FC01E25AF84F81818D7FA5
:1034D000818349C1981798F085E08983F901E25A00
:1034E000F84F80818064808321E0AE014F5F5F4FA1
:1034F00060E08C2D0E94A50E84E0F80130C090E0C1
:10350000F801438950E04F5F5F4F6189460F511DBD
:10351000841795072CF1F901E25AF84F808182FF58
:1035200015C083E089838BE18C9DF0018D9DF00DAA
:103530001124E25AF84F81818E7F818321E0AE0110
:103540004F5F5F4F60E88C2D0E94A50E8BE18C9D34
:10355000F0018D9DF00D1124EB5BF84F81E083832A
:103560008BE18C9DF0018D9DF00D1124DF01AB5B93
:10357000B84F14969C91149713968C9113979817A3
:1035800079F011969C91119751968C91981740F073
:1035900082E08983E25AF84F818182608183B9C0D9
:1035A0002BE12C9DC0012D9D900D1124FC01EB5BA6
:1035B000F84F618170E0218930E0448950E073CF99
:1035C000F8019185418183896089992309F45EC05E
:1035D000042E000C550B082E000C990B0196860F3B
:1035E000911D67FD9A9548175907E4F0F901E25AD1
:1035F000F84F808180FF0CC095E099838F7B80839A
:1036000021E0AE014F5F5F4F60E88C2D0E94A50E58
:103610008BE18C9DF0018D9DF00D1124EB5BF84F3B
:1036200082E083838BE18C9DF0018D9DF00D112450
:10363000DF01AB5BB84F14969C91149713968C9155
:103640001397981741F011969C91119750968C9171
:1036500098170CF057C08BE18C9DF0018D9DF00DFB
:103660001124DF01AB5BB84F11964C911197042EDA
:10367000000C550B51968C915197082E000C990B0C
:1036800054962C91022E000C330B5DC050E090E05C
:103690000196860F911D48175907E4F0F901E25A87
:1036A000F84F808180FF0CC095E099838F7B8083E9
:1036B00021E0AE014F5F5F4F60E88C2D0E94A50EA8
:1036C0008BE18C9DF0018D9DF00D1124EB5BF84F8B
:1036D00082E083838BE18C9DF0018D9DF00D1124A0
:1036E000DF01AB5BB84F14969C91149713968C91A5
:1036F00013979817A1F011969C91119750968C9161
:10370000981768F084E08983E25AF84F80818068D6
:10371000808321E0AE014F5F5F4F60E029C08BE105
:103720008C9DF0018D9DF00D1124DF01AB5BB84F36
:1037300011964C91119750E051968C91519790E0D1
:1037400054962C9130E02F5F3F4F821B930B8417D0
:1037500095078CF0E25AF84F808187FF0CC094E007
:1037600099838F77808321E0AE014F5F5F4F60E8E0
:103770008F2D0E94A50E8BE18C9DF0018D9DF00D8B
:103780001124EB5BF84F838184830F90DF91CF91FD
:103790001F910F91FF90EF90DF90CF9008956111EE
:1037A00002C022E001C023E0FC01208321E021834C
:1037B00082E00895CF93DF93F901DC018D919C9114
:1037C00084309105E8F54D33D8F56134C8F5833080
:1037D000910561F0A42FB0E0A60FB11DEC01CF5709
:1037E000D84F288130E02A173B0754F19C012F5F06
:1037F0003F4F2330310528F421E0280F2083118228
:1038000006C02FEF2083218383309105D9F0262F26
:1038100030E0DF011296880F991FFC01E558F84F40
:10382000822F861B841748F4C081D181C20FD31F19
:1038300088818D932F5F3F4FF3CF82E0840F03C0C9
:103840008FEF01C082E0DF91CF910895CF93DF9396
:10385000FB01282F30E0233031050CF073C082309B
:1038600008F072C08BE1829FD001839FB00D1124BC
:10387000AB5BB84F1896CC911897D0E0CC0FDD1FFA
:10388000C558D84F0990D881C02D8B81813009F05F
:1038900051C08FE380831896CC911897D0E0CC0F5D
:1038A000DD1FC558D84F0990D881C02D89A58183C7
:1038B0001896CC911897D0E0CC0FDD1FC558D84F83
:1038C0000990D881C02D88A582831896CC9118972D
:1038D000D0E0CC0FDD1FC558D84F0990D881C02D3E
:1038E0008FA183831896CC911897D0E0CC0FDD1F61
:1038F000C558D84F0990D881C02D8EA184831896C1
:10390000CC911897D0E0CC0FDD1FC558D84F099047
:10391000D881C02D8DA185831896AC91B0E0AA0FF7
:10392000BB1FA558B84F0D90BC91A02D94968C91BB
:1039300086830AC010821182128213821482158239
:10394000168202C08FEF01C087E0DF91CF9108950A
:10395000AF92CF92EF920F93E82FF0E0E330F105B2
:103960000CF08EC0823008F089C08BE18E9FD001B0
:103970008F9FB00D1124AB5BB84F1896AC91B0E09F
:10398000AA0FBB1FA558B84F0D90BC91A02D139640
:103990008C911397813009F071C060FF02C0999635
:1039A0004C9361FF14C08BE18E9FD0018F9FB00DAF
:1039B0001124AB5BB84F1896AC91B0E0AA0FBB1FB7
:1039C000A558B84F0D90BC91A02D98962C9362FFEE
:1039D00014C08BE18E9FD0018F9FB00D1124AB5B83
:1039E000B84F1896AC91B0E0AA0FBB1FA558B84FBE
:1039F0000D90BC91A02D97960C9363FF14C08BE1A2
:103A00008E9FD0018F9FB00D1124AB5BB84F1896DD
:103A1000AC91B0E0AA0FBB1FA558B84F0D90BC9158
:103A2000A02D9696EC9264FF14C08BE18E9FD0017E
:103A30008F9FB00D1124AB5BB84F1896AC91B0E0DE
:103A4000AA0FBB1FA558B84F0D90BC91A02D9596FD
:103A5000CC9265FF13C02BE12E9FC0012F9F900DCC
:103A60001124FC01EB5BF84FE085F0E0EE0FFF1F47
:103A7000E558F84F0190F081E02DA4A280E001C04C
:103A80008FEF0F91EF90CF90AF900895FB0190E0F2
:103A90008330910564F52BE1289FD001299FB00D5B
:103AA0001124AB5BB84F15962C911597223F11F45A
:103AB000108203C011962C9120832BE1289FD00106
:103AC000299FB00D1124AB5BB84F16968C911697B9
:103AD000818315968C911597823F19F411968C91DC
:103AE00002C013968C918283138284E008958FEF35
:103AF0000895811109C080912707FB01808380917F
:103B00002807818382E008958FEF08952BE1829F3B
:103B1000C0011124FC01EB5BF84F618308952BE198
:103B2000829FC0011124FC01EB5BF84F8181089555
:103B30002BE1829FC0011124FC01EB5BF84F81E077
:103B4000828308952BE1829FC0011124FC01EB5B6D
:103B5000F84F8281128208952BE1829FC0011124C7
:103B6000FC01EB5BF84F858108952BE1829FC0013A
:103B70001124FC01EB5BF84F878108950E949A1E87
:103B800080E00E941A058093610780914B07803C7A
:103B900041F480914A078150823018F480E00E94FD
:103BA0007B1580916607803C41F4809165078150C8
:103BB000823018F481E00C947B150895039666E139
:103BC00070E00E949B1E8CE0869F9001879F300DC5
:103BD000112480E090E08217930719F0000001960D
:103BE000FACF0895039666E170E00E949B1E8CE078
:103BF000869FA001879F500D112428EE33E080E0BE
:103C000090E08417950719F000000196FACF215033
:103C10003109A9F7089593B7987F892B83BF089539
:103C2000109285071092840710926F0210926E0214
:103C300010926D0210926C0210926B0283B7886032
:103C400083BF83E00E940B1E12BE8CE881BF87B742
:103C5000826087BF08951F920F920FB60F921124B2
:103C60000BB60F922F933F934F935F936F937F9376
:103C70008F939F93AF93BF93EF93FF9380916D02C8
:103C800090916E02019690936E0280936D02209146
:103C90006B0230916C022F5F3F4F30936C02209388
:103CA0006B02099734F010926E0210926D020E941E
:103CB000CB1380916B0290916C02843691053CF09D
:103CC00081E080936F0210926C0210926B02FF9160
:103CD000EF91BF91AF919F918F917F916F915F9184
:103CE0004F913F912F910F900BBE0F900FBE0F90F1
:103CF0001F90189580916F0210926F0208959C0199
:103D000090E0615030F0F901E60FF11D8081980FCD
:103D1000F8CF892F81950895CF93C42F0E947F1EDD
:103D2000C81B8C2FCF910895089581E0089581E0FC
:103D3000089508950895AA1BBB1B51E107C0AA1F4F
:103D4000BB1FA617B70710F0A61BB70B881F991F3C
:103D50005A95A9F780959095BC01CD010895EE0F75
:103D6000FF1F0024001C0BBE0790F691E02D099464
:103D70000F931F93CF93DF938230910510F482E06D
:103D800090E0E0918A07F0918B0720E030E0A0E01E
:103D9000B0E0309719F140815181028113814817B9
:103DA0005907C8F08417950769F4109731F01296F7
:103DB0000C93129713961C9327C000938A071093B5
:103DC0008B0722C02115310519F04217530718F44B
:103DD0009A01BD01EF01DF01F801DBCF21153105AB
:103DE000F9F0281B390B2430310580F48A819B813E
:103DF0006115710521F0FB019383828304C09093C8
:103E00008B0780938A07FE01329644C0FE01E20FC1
:103E1000F31F8193919322503109398328833AC04B
:103E20002091880730918907232B41F420910201CA
:103E30003091030130938907209388072091000176
:103E4000309101012115310541F42DB73EB7409164
:103E5000040150910501241B350BE0918807F09176
:103E60008907E217F307A0F42E1B3F0B2817390729
:103E700078F0AC014E5F5F4F2417350748F04E0FC6
:103E80005F1F50938907409388078193919302C0E5
:103E9000E0E0F0E0CF01DF91CF911F910F91089505
:103EA000CF93DF93009709F481C0FC01329713820E
:103EB0001282A0918A07B0918B07109781F420811C
:103EC0003181820F931F209188073091890728172D
:103ED000390751F5F0938907E093880767C0ED0132
:103EE00020E030E0CE17DF0740F44A815B819E017D
:103EF00041155105F1F0EA01F5CFD383C28340812A
:103F00005181840F951FC817D90759F48881998169
:103F1000840F951F0296918380838A819B8193836E
:103F200082832115310529F4F0938B07E0938A07EA
:103F30003DC0E901FB83EA8349915991C40FD51F24
:103F4000EC17FD0761F480819181840F951F029623
:103F5000E90199838883828193819B838A83E0E04E
:103F6000F0E012968D919C911397009719F0FD0146
:103F7000DC01F7CF8D919C9111979D012E5F3F4FF2
:103F8000820F931F209188073091890728173907DE
:103F900069F4309729F410928B0710928A0702C0B7
:103FA00013821282B0938907A0938807DF91CF9183
:063FB0000895F894FFCF14
:103FB60000008C072000FF0300510137000000C1FC
:103FC6000003C1F26F070000000700C000000000F8
:103FD60000000000000000000000000000000000DB
:103FE600000000000000CC414D4320484F545F5371
:103FF6005741500000510100000001C1007FFC0242
:1040060001FF7FFF7F0000000400004D0240010019
:10401600DE079AB481FF00F5CEB481674D0606002F
:104026000000C331325644554E455F57524D434802
:104036000030303030303030303100436F726546FA
:104046005255004345524E204D4D430044554E4572
:0C4056005F5444455F57524D4348000042
:00000001FF
